:1000000010C02AC06CC128C027C026C09FC124C010
:1000100023C022C021C020C01FC01EC01DC01CC0E4
:100020001BC011241FBECFE5D1E0DEBFCDBF10E065
:10003000A0E6B0E0EEECF7E002C005900D92A43728
:10004000B107D9F721E0A4E7B0E001C01D92A830C4
:10005000B207E1F7A4D0B9C3D3CF982F96959827CC
:10006000892F869586958927982F92959F70892745
:10007000089510927C0089B3887390E033E09595E1
:1000800087953A95E1F780936A0090916900809195
:100090006A00981709F444C080916A00809369004F
:1000A0008091FB009091FC0080FF06C080916A0067
:1000B0008095877080936A008091FB009091FC008E
:1000C00081FF05C080916A00C8DF80936A0080913B
:1000D0006A0090E0880F991F079673D390930701E9
:1000E00080930601809106019091070162D380936D
:1000F00074004091740060910601709107016F5F78
:100100007F4F50E080E890E045D380E197E2909304
:1001100068008093670083B5816083BD1DBC1CBCF3
:100120008091010190910201892BC9F02091670013
:1001300030916800809101019091020128173907E0
:1001400074F0109268001092670081E080937C0048
:100150001092FE001092FD0010927D0017C0809159
:10016000800090E09093FE008093FD0089B387703B
:1001700080937D008091FB009091FC0080FF06C081
:1001800080917D008095877080937D00E0917D0057
:10019000F0E0E559FF4F808180930301089580E0EE
:1001A00090E007D3C82F843009F098C081E090E038
:1001B00008D39093FC008093FB008091FB0090910A
:1001C000FC00807F992754E0969587955A95E1F732
:1001D00068E572E0CDD2909302018093010183E043
:1001E00090E0EFD2909305018093040185E090E0C8
:1001F000E8D290937F0080937E008BEF88BBC7BBD3
:100200008FE78BBB80E88ABB8FB580688FBD619A12
:1002100082E083BFE0E0F0E089E080935700E49162
:10022000EF70E23051F48EB58D608EBD8DE486BFE7
:1002300081E690E09BBD8ABD4EC08091FB0090910D
:10024000FC00892F990F990B8770992782309105AF
:10025000E9F02CF4009751F00197C9F50FC08430F4
:10026000910521F1DCF0059791F528C08FE486BF58
:100270008EB58D608EBD83E690E027C083EB86BF90
:100280008EB58D608EBD80EE90E01FC08CE786BF7E
:100290008EB58B608EBD83EC99E017C081E686BF7A
:1002A0008EB58A608EBD88E09DE30FC08DE486BF69
:1002B0008EB58A608EBD83ED90E307C08CE986BF62
:1002C0008EB58B608EBD84E39CE09BBD8ABD80E1D2
:1002D0008BBF80E482BBCDDE7894FFCFFFCF1F922F
:1002E0000F920FB60F9211248F939F93CE9B27C02E
:1002F00080916100909162000197909362008093D9
:100300006100892BE1F480917E0090917F009093B1
:1003100062008093610080917900882381F081E000
:1003200090E0909364008093630081E08093780074
:100330001092790083B5816083BD1DBC1CBC9F9168
:100340008F910F900FBE0F901F9018951F920F92D4
:100350000FB60F9211242F933F934F935F936F9398
:100360007F938F939F93AF93BF93CF93DF93EF933D
:10037000FF9380917700982F91509093770081118F
:10038000E4C180917600809377008091670090911E
:1003900068000196909368008093670080916300E5
:1003A0009091640001979093640080936300892B7F
:1003B00029F080917800882391F0C7C180910401D1
:1003C0009091050190936400809363008091780080
:1003D000882319F081E080930301109278008091C6
:1003E0007500893B21F0809175008A3B21F4809152
:1003F00079008111AAC180917A0090917B00892BAC
:1004000079F080917A0090917B00019790937B0026
:1004100080937A00892B09F098C181E080930301D1
:100420008091030181508093030181118EC1E0917D
:100430007D00F0E0E559FF4F8081809303018091BA
:1004400075008938E1F0809175008838C1F080919D
:1004500075008039A1F0809175008F3881F080910E
:1004600075008A3861F0809175008B3841F0809179
:100470007500893B21F0809175008A3B49F486EF35
:10048000809366008FEF809365008FEE809360000D
:100490008091660081508093660087FF3CC1809107
:1004A000650087FF8DC0809175008F3E29F4809193
:1004B00066008A3F0CF049C1809166008E3F0CF4C3
:1004C0007FC043C1D6DD809174002091FD00309142
:1004D000FE0090E0019728173907A4F78091FD00EE
:1004E0009091FE00FC01E058FF4F218120937500A0
:1004F00001969093FE008093FD0080917500887FA7
:10050000803899F480917C0081110DC08091750034
:10051000877080937D00E0917D00F0E0E559FF4F0A
:10052000808180930301109275008091750088236B
:1005300051F2809175008D3859F48091FB009091B3
:10054000FC008C709927089709F4C298C093750035
:10055000809175008E3859F48091FB009091FC00D9
:100560008C709927089709F4C29AC09375008091FE
:10057000FB009091FC008C709927049739F48091CE
:100580007D00882311F0C29801C0C29AD093650003
:1005900005C0809165008150809365008091750051
:1005A0002091650090E002C0959587952A95E2F725
:1005B00080FDEFCF8091650081508093650002C07F
:1005C000CBEBD7E08091650087FD7DCF80917C00EB
:1005D000882339F0809175008A3819F48FEE809362
:1005E0007500809175008F3809F450C088F48938FF
:1005F00059F138F48C3709F452C0883809F071C0C9
:1006000027C08A3809F455C08B3809F06AC057C032
:100610008A3B09F45EC030F48039A1F1893B09F0CE
:1006200060C053C08B3B09F45AC08F3E09F059C0DB
:10063000809160008F3E19F41092660003C08DEF28
:10064000809366008FEF61C081E08093660002C0F6
:10065000109266002091FD003091FE00F901E058F3
:10066000FF4F818190E06AE070E082D00197909323
:100670007B0080937A002F5F3F4F3093FE002093E2
:10068000FD0045C081E08093660002C010926600C4
:1006900089E090E090937B0080937A0038C085B722
:1006A000877E806185BFF89485B7806285BF889515
:1006B0002EC081E0809378001092660028C081E00F
:1006C000809378008093660022C01092660081E0DB
:1006D00003C081E0809366008093790018C086EFA4
:1006E000AFCF809175002091650090E002C0959594
:1006F00087952A95E2F780FF02C083E001C081E080
:1007000080936600809165008150809365008091A0
:100710007500809360008091660018165CF4DF9A83
:100720008091FB009091FC008C709927892B69F4D3
:1007300082E40AC0DF988091FB009091FC008C70ED
:100740009927892B11F482E080BFFF91EF91DF910F
:10075000CF91BF91AF919F918F917F916F915F9159
:100760004F913F912F910F900FBE0F901F901895B2
:100770005527002480FF02C0060E571F660F771F03
:100780006115710521F096958795009799F7952F3A
:10079000802D0895DC01862FE82FE199FECF1FBA46
:1007A00005C0EEBBE09AE3950DB20D924150C8F73B
:1007B0000895E199FECF1FBA8EBBE09A99278DB3B9
:0E07C0000895A8E1B0E042E0E7CFF894FFCF43
:1007CE00EF01000100FFF61027626301020A1E3CD2
:0407DE0064962C00F1
:00000001FF
